:1000000012C019C018C017C016C015C014C013C044
:1000100012C011C010C00FC00EC00DC00CC00BC06C
:100020000AC009C008C011241FBECFE5D4E0DEBF5E
:10003000CDBF66D067C0E4CF80B38095817008954E
:1000400080B38695817091E08927089580B382FB03
:10005000882780F991E08927089580B383FB88275A
:1000600080F991E089270895E7DF81110CC0E8DF6E
:1000700081110CC0EBDF81110CC0EFDF81110CC0CE
:1000800080E090E008958AE090E0089584E190E0B7
:10009000089582E390E0089584E690E0089580B3A7
:1000A0008295817091E08927089520E030E04FEF3C
:1000B00028173907BCF448BB5FE76AE176E0515086
:1000C00060407040E1F700C0000018BA5FE76AE1E5
:1000D00076E0515060407040E1F700C000002F5FB3
:1000E0003F4FE6CF0895C0DFEC01D9DF8823D9F375
:1000F000CE01DBDFF8CF8FEF87BB11BA82BB08954B
:08010000FADFF1DFF894FFCFF4
:00000001FF
